:100000000C94F4020C94C4040C9411030C9411038A
:100010000C9411030C9411030C9411030C94110310
:100020000C9411030C9411030C9411030C94110300
:100030000C9411030C9411030C9411030C941103F0
:100040000C9411030C9411030C9411030C941103E0
:100050000C9411030C9411030C9411030C941103D0
:100060000C9411030C941103040309041803720087
:100070006100700068006E00650074002E006E0064
:10008000650074002803470043002F004E0036002F
:100090003400200074006F0020005500530042001F
:1000A0002C002000760032002E00330012011001D7
:1000B000000000089B28040003020102030109025A
:1000C0002200010100803209040000010300000049
:1000D00009210101000122EC040705810308000544
:1000E0000A0330003000300031001201010100002D
:1000F00000089B2804000302010203010501090511
:10010000A10185010901A1000501750895061500E9
:1001100026FF00350046FF00093009310933093454
:10012000093509368102050915002501750195106B
:1001300019012910750195108102C0050F0992A1BE
:10014000028502099F09A009A409A509A615002591
:100150000135004501750195058102950375018101
:1001600003099415002501350045017501950181AC
:1001700002092215012528350145287507950181B9
:1001800002C00921A1028501092215012528350196
:1001900045287508950191020925A102092609271C
:1001A000093009310932093309340940094109424A
:1001B00009430928250C15013501450C75089501E1
:1001C0009100C0095009540951150026FF7F3500E0
:1001D00046FF7F66031055FD75109503910255008B
:1001E0006600000952150026FF00350046102775ED
:1001F0000895019102095315012508350145087537
:1002000008950191020955A102050109300931152E
:10021000002501750195029102C0050F095695014F
:100220009102950591030957A1020B01000A000BE9
:1002300002000A0066140055FE150026FF00350076
:1002400047A08C00006600007508950291025500D9
:10025000660000C0050F09A766031055FD150026AE
:10026000FF7F350046FF7F75109501910266000003
:100270005500C0050F095AA1028502092215012562
:100280002835014528750895019102095B095D151E
:100290000026FF00350046102795029102095C09EF
:1002A0005E66031055FD26FF7F46FF7F75109102A5
:1002B00045006600005500C0095FA10285030922C0
:1002C0001501252835014528750895019102092356
:1002D0001500250135004501750495019102095865
:1002E000A1020B01000A000B02000A007502950230
:1002F0009102C01580257F36F0D846102709607519
:10030000089501910236F0D84610270961096295D7
:10031000029102150026FF003500461027096309E7
:1003200064750895029102096546102795019102AE
:10033000C0096EA102850409221501252835014551
:10034000287508950191020970150026FF003500F7
:10035000461027750895019102096F1580257F3693
:10036000F0D846102795019102097166140055FED8
:10037000150026FF00350047A08C0000910209728D
:1003800026FF7F46FF7F66031055FD75109501918E
:10039000026600005500C00973A1028505092215F7
:1003A0000125283501452875089501910209701627
:1003B00001FF26FF0036F0D84610277510950191F1
:1003C00002C00974A10285060922150125283501FC
:1003D0004528750895019102097509761580257FD4
:1003E00036F0D8461027750895029102C00968A119
:1003F000028507092215012528350145287508952C
:10040000019102096C15002610273500461027754A
:10041000109501910209691581257F350046FF007D
:100420007508950C920201C00966A10285080501B4
:10043000093009311581257F350046FF0075089583
:10044000029102C0050F0977A102850A0922150150
:100450002528350145287508950191020978A102E2
:100460000979097A097B1501250375089501910021
:10047000C0097C150026FF00350046FF009102C030
:100480000990A102850B092225281501350145286F
:10049000750895019102C00996A102850C0997097A
:1004A000980999099A099B099C15012506750895D3
:1004B000019100C0097DA102850D097E150026FF6E
:1004C000003500461027750895019102C0096BA1FF
:1004D00002850E0922150125283501452875089544
:1004E000019102096D150026FF00350046FF0075D9
:1004F0000895019102095166031055FD150026FF6C
:100500007F350046FF7F751095019102550066000A
:1005100000C009ABA10285090925A1020926092706
:1005200009300931093209330934094009410942C6
:1005300009430928250C15013501450C750895015D
:10054000B100C00501093B150026FF01350046FF3B
:1005500001750A9501B1027506B101C0050F09893F
:10056000A1028502092225281501350145287508B3
:100570009501B102098BA102098C098D098E250311
:1005800015013501450375089501B100C009AC1589
:100590000027FFFF0000350047FFFF0000751095A2
:1005A00001B100C0097FA102850309807510950182
:1005B0001500350027FFFF000047FFFF0000B102D4
:1005C000098326FF0046FF0075089501B10209A9BD
:1005D00009AA750195021500250135004501B102F2
:1005E00075069501B103C0C011241FBECFEFD4E042
:1005F000DEBFCDBF11E0A0E0B1E0E4E4FAE102C06B
:1006000005900D92A033B107D9F712E0A0E3B1E055
:1006100001C01D92AC3AB107E1F70E944E070C945D
:10062000200D0C940000E9E6F0E080818260808378
:10063000E89A8BE480937E018AE580937D0108959A
:100640001F93CF93DF9360918E01635067FDDDC0F0
:1006500080918B01CCE0D0E0C81BD109CE56DE4F93
:1006600080918A018D3209F0BBC0683009F0CBC09F
:1006700083EC809372018AE580930001109230012F
:100680008881807629F0CE010E946A06AC0190C074
:100690009A8110927B018981882329F410927C0130
:1006A00042E050E07EC0853019F490938F0177C00E
:1006B000863009F05EC08B81813049F48CEA90E08D
:1006C00090938D0180938C0142E150E04EC08230C6
:1006D00049F48EEB90E090938D0180938C0142E27F
:1006E00050E043C0833069F58A81882349F488E665
:1006F00090E090938D0180938C0144E050E035C0F0
:10070000813049F48CE690E090938D0180938C01C8
:1007100048E150E02AC0823049F484E890E09093A8
:100720008D0180938C0148E250E01FC08330D9F4E2
:1007300080EE90E090938D0180938C014AE050E030
:1007400014C0813249F480ED90E090938D01809344
:100750008C0149E050E009C0823229F4CE010E94A8
:10076000FE05AC0102C040E050E080E4809330011F
:100770001FC0883029F441E050E021E931E013C086
:10078000893019F4909391010AC08A3019F441E03C
:1007900050E007C08B3019F48BE480937E0140E079
:1007A00050E02BE731E030938D0120938C010DC098
:1007B0002FEF4F3F520749F4888187FF02C04E81D7
:1007C0005F8180E88093300106C08E819F8184170D
:1007D000950708F4AC01509302014093010113C046
:1007E0008091300187FF0FC0CE010E94CE068F3F5F
:1007F00021F48EE18093000106C0882321F010923D
:1008000002011092010110928E018091000184FF7B
:1008100061C08091010190910201EFEF8F3F9E072F
:1008200009F458C09C018930910510F028E030E0AF
:10083000821B930B909302018093010180917201BE
:1008400098E8892780937201122F222391F16091F9
:100850008C0170918D018091300186FF13C09B0146
:10086000C3E7D1E01150412F50E01F5FDA01AC58CF
:10087000BE4FF901849189932F5F3F4FCA17DB0761
:10088000C1F70FC0DB01E3E7F1E01150412F50E069
:100890001F5F9A012C583E4F8D918193E217F30709
:1008A000D9F7CA010196860F971F90938D01809307
:1008B0008C0183E791E0612F0E94C004612F6C5F7F
:1008C0006C3031F08FEF9FEF909302018093010124
:1008D0006093000194E189B1857031F49150D9F7AA
:1008E00010928F0110928901DF91CF911F9108958D
:1008F0001F93DC01162F80917D0184FF07C080913A
:100900007E0198E8892780937E0103C08AE5809361
:100910007D01912FEFE7F1E08D91819391501916B0
:10092000DCF38FE791E0612F0E94C0041C5F1093FD
:100930007D011F910895A82FB92F8FEF9FEF1BC046
:100940002D918227282F22952827722F26952695CC
:100950002727239526952170782F892F8227219587
:10096000207C922F222776952795972782277695A8
:10097000279597278227615018F7809590950895BD
:10098000DADF8D939D930895CF93CFB7CF93C3951F
:10099000489BE9F7489B09C0489B07C0489B05C096
:1009A000489B03C0489B01C0A3C0DF93C0918B014B
:1009B000DD27CE56DE4F489B02C0DF91EBCF2F9351
:1009C0000F931F9309B12FEF00FB20F94F933F9333
:1009D00019B14FEF012700FB21F93BE031C04E7FF9
:1009E000012F19B1216028C0102F4D7F2260000017
:1009F00009B129C04B7F2460012F000019B12BC021
:100A000019B1477F28602AC04F7E09B120612CC0F0
:100A10004F7D19B120622FC04F7B09B1206432C0D5
:100A2000422709B149934FEF0000102710FB20F92E
:100A300019B11570C9F1297F91F2012700FB21F945
:100A400009B1237F89F2315058F1102710FB22F9A8
:100A500019B1277E79F2012700FB23F92F7C81F25F
:100A600009B1102710FB24F92F7971F200C019B1D8
:100A7000012700FB25F92F7359F200C009B1102797
:100A800010FB26F9223040F200C019B1012700FB0B
:100A900027F9243028F64F77206819B10000F9CFE4
:100AA00011E01CBB002719C03B503195C31BD0403F
:100AB00011E01CBB0881033CF9F00B34E9F02091F4
:100AC00089011981110F1213EDCF4A81441F093694
:100AD00041F10D3211F0013E29F7009390013F9151
:100AE0004F911F910F912F91DF91CCB3C0FD4FCF4C
:100AF000CF91CFBFCF91189520919001222379F308
:100B000010918E01112369F534306AF130938E0112
:100B100020938A0110918B013BE0311B30938B01B4
:100B200022C000918E010130E4F40AE54F7049F4CF
:100B30003091000134FD19C000930001C2E7D1E0FB
:100B400018C030917D0134FD10C000937D01CEE7C7
:100B5000D1E00FC02795A8F45150A9F4220F00004E
:100B6000F9CF4AE503C042ED01C0432FC4E1D0E014
:100B700032E01AB11560589A1AB90BB120E415E0A9
:100B80005F93012756E00BB9279520F4515021F4CB
:100B9000220FF9CF012756E000003B5A0BB9D0F2E3
:100BA000279528F4515029F4220F0000F9CF01278E
:100BB00056E027950BB920F4515021F4220FF9CFBC
:100BC000012756E0299133230BB921F60A7F1091B2
:100BD0008F01110FC651D0400BB911F0109389014C
:100BE00011E01CBB01601AB11A7F402F4A7F5F9150
:100BF00000C000C00BB91AB94BB971CFFC0180819C
:100C0000807619F58181863001F58381813019F074
:100C10008232D9F40DC080913501909136019093C4
:100C20008D0180938C0180913701282F30E00FC017
:100C3000809131019091320190938D0180938C01CC
:100C4000209133013091340102C020E030E0C9012D
:100C50000895E0913801F0913901309749F0028808
:100C6000F389E02D309721F0992787FD909509951C
:100C70000895DC01E0913801F0913901309719F5C0
:100C80006130710519F020E030E022C081E08C93E2
:100C90008FE711968C93119712968C931297139657
:100CA0008C93139714968C93149715968C93159791
:100CB00016968C93169717961C92179718961C9257
:100CC00029E030E005C00088F189E02D09959C01FC
:100CD000C9010895FC014DE351E050938D0140930B
:100CE0008C01808180768032B9F52181213019F024
:100CF000293091F52EC08381813019F0833049F578
:100D000009C06281662329F1CA0170E00E94390698
:100D10009C0124C06281623061F460933D012093A4
:100D20003E0120933F018AE080934001809341017E
:100D30000DC0633071F460933D0120933E01209318
:100D40003F018FEF809340012093410125E030E087
:100D500005C02FEF3FEF02C020E030E0C901089549
:100D60008091480190914901892B11F410923A0128
:100D700080913A01882319F40E94290608958091F0
:100D80003B0187FF03C081E00E94290680913C015E
:100D900087FF03C081E00E9429060895FC016623B5
:100DA00009F449C08081853089F0863030F4813083
:100DB00049F0843009F03FC010C0893019F08A3002
:100DC000D1F50FC081818093470135C08181813089
:100DD00091F5828180933B012CC0828180933C01FC
:100DE00028C0643041F5838190E023E0880F991F8B
:100DF0002A95E1F79093490180934801818190E021
:100E00008F7790708130910531F0813091059CF0A1
:100E10000397029780F48281823029F0833039F081
:100E2000813049F401C081E080933A0102C0109200
:100E30003A010E94B00681E008950F931F93CF936B
:100E4000DF93BC0180917D0184FF23C08DE391E09D
:100E50000E943906C0E0D0E0082F112707FD109549
:100E600015C00E942003A89580917D0184FFF9CFD1
:100E7000CE01835C9E4FB8016C1B7D0B6930710500
:100E800014F068E070E00E9478042896C017D1073B
:100E90005CF3DF91CF911F910F9108954F925F9274
:100EA0006F927F928F929F92AF92BF92CF92DF927A
:100EB000EF92FF920F931F93DF93CF9300D0CDB7A4
:100EC000DEB71A82198281E084B98EEF85B917B82E
:100ED0008FEF88B988EF8BB985E08AB914BC85BDDE
:100EE00082E08093B00087E08093B10082E380933A
:100EF000B3008CEF90E090933201809331010E9417
:100F0000090D90933401809333018AEE90E0909321
:100F10003601809335010E94060D809337018BB115
:100F20008A7F8BB98AB185608AB988EC9FEA01977C
:100F3000F1F78AB18A7F8AB90E94C9082FE088E157
:100F400090E00FB6F894A895809360000FBE2093B0
:100F500060000E9413037894BB24AA24A394EE2477
:100F6000FF244424439452E0552E4CE2842E41E069
:100F7000942E31E0632E712C04C0BB2402C0EE24F9
:100F8000FF24A8952FE1E216F10424F01092390114
:100F9000109238018091380190913901892B09F024
:100FA00069C080E00E9429060E94200381E090E051
:100FB0000E941D078CE291E0F4013197F1F701974F
:100FC000D9F70E9420030E947A098230910541F0EE
:100FD00083309105A1F0019791F60E94F80C02C0B0
:100FE0000E943C0BFC0190933901809338010284EC
:100FF000F385E02D099580E00E942906C0CF0E946C
:101000003C0BFC0190933901809338010284F385F5
:10101000E02D0995E0913801F09139010488F589B6
:10102000E02D0995882309F50E94200380E991E0CD
:10103000F4013197F1F70197D9F70E9420030E943C
:10104000F80CFC0190933901809338010284F385F8
:10105000E02D0995E0913801F09139010488F58976
:10106000E02D0995882309F48ACF80E00E942906A3
:10107000EE24FF24A8950E942003AA20A1F00E943C
:10108000B006E0913801F09139010484F585E02D36
:101090000995882321F4AA24EE24FF2404C008948F
:1010A000E11CF11CAA24B99B3FC057BABB2009F030
:1010B0003BC00E94B00683B7816083BF889583B729
:1010C0008E7F83BFC4010197F1F7E0913801F09161
:1010D00039010484F585E02D0995882319F4EE245F
:1010E000FF2403C00894E11CF11C00E010E013C0D1
:1010F00068010894C11CD11C0684F785E02DC60147
:101100000995882339F0C30102C0880F991F0A95F9
:10111000E2F7B82A8601E0913801F0913901848123
:1011200095810817190724F3A89B10C045BA809130
:10113000480190914901009749F02FEF8F3F9207A6
:1011400029F001979093490180934801BB2009F44D
:1011500018CF00E010E0CB2CDD24C7FCD0940FC0EA
:10116000C601002E02C0959587950A94E2F780FF8C
:1011700004C0C80101960E941D070F5F1F4FE09138
:101180003801F0913901848195810817190744F3DA
:10119000F4CE3D984598249A2C980895EF92FF92AA
:1011A0000F931F93CF93DF937C01662309F44FC005
:1011B00070E020E030E0E0E0F0E011C088818423BE
:1011C000FD01E855FE4F808311964695A017B107A3
:1011D000A9F72F5F3F4F2617370754F4FD01DF01B2
:1011E00040E8E701C20FD31F8F01085F1F4FE6CF12
:1011F000E8EAF1E0CF93DF93EF93FF9301910023AF
:1012000011F049F416C000003D9A19E00FD03D9846
:101210001197A1F70EC03D9A11E008D03D9815E056
:1012200005D000000000119749F703C01A95F1F7A7
:1012300008950000FF91EF91DF91CF913D9A11E069
:10124000F5DF3D980FEF0A9511F0359BFCCFE8EAEA
:10125000F1E0EF93FF93112700270395A1F0359953
:10126000FCCF08C004E6039572F03599FCCF1395C6
:1012700051F0019304E6039532F0359BFCCF1395B2
:1012800011F00193EFCFFF91EF91612F70E06115A5
:10129000710531F110FF24C040E050E020E030E063
:1012A0000CC08081F901E955FE4F9081E0E089177B
:1012B00008F4E1E0EC934F5F5F4FDA01A855BE4FB1
:1012C000F901E855FE4F2E5F3F4F411750F384E17F
:1012D0008A95F1F79B01215030403595279502C042
:1012E00020E030E0C901DF91CF911F910F91FF9075
:1012F000EF900895DF93CF930F92CDB7DEB71982A9
:10130000CE01019661E070E00E94CE08009719F4CA
:1013100020E030E026C0489711F58091AC01882389
:1013200011F098E001C090E08091AD0181119460CE
:101330008091AE01811192608091AF018111916025
:101340009A3028F4983028F4953049F405C09B3041
:1013500031F422E030E005C021E030E002C023E0BB
:1013600030E0C9010F90CF91DF91089590934B0128
:1013700080934A010895009741F0DC01EEE4F1E02A
:1013800089E001900D928150E1F7A7E5B1E0EEE42C
:10139000F1E089E001900D928150E1F789E090E061
:1013A00008958EE491E067E571E049E050E00E9425
:1013B0000C0D08950F931F93DF93CF93CDB7DEB736
:1013C00029970FB6F894DEBF0FBECDBF1982CE01AC
:1013D000019661E070E00E94CE08883109F020C1DA
:1013E00080E48A8383E08B831C8280914A01909100
:1013F0004B01892B11F081E08C838E010E5F1F4F12
:10140000C80163E070E00E94CE08803409F008C192
:1014100088E0F80111928A95E9F74A8120E030E0EE
:1014200060E870E0F901E854FE4F8081882339F0CC
:10143000CB01022E02C0959587950A94E2F7482BBE
:101440002F5F3F4F2830310569F74A834B8120E0F9
:1014500030E060E870E0F901E054FE4F80818823BD
:1014600039F0CB01022E02C0959587950A94E2F7D8
:10147000482B2F5F3F4F2830310569F740954B834C
:101480004C8120E030E060E870E0F901E853FE4F65
:101490008081882339F0CB01022E02C09595879573
:1014A0000A94E2F7482B2F5F3F4F2830310569F748
:1014B0004C834D8120E030E060E870E0F901E053BA
:1014C000FE4F8081882311F080E007C0CB01022EFF
:1014D00002C0959587950A94E2F7482B2F5F3F4FFE
:1014E0002830310559F74D834E8120E030E060E827
:1014F00070E0F901E852FE4F8081882339F0CB017A
:10150000022E02C0959587950A94E2F7482B2F5F2B
:101510003F4F2830310569F740954E834F8120E0D9
:1015200030E060E870E0F901E052FE4F80818823EE
:1015300039F0CB01022E02C0959587950A94E2F707
:10154000482B2F5F3F4F2830310569F740954F8377
:10155000488520E030E061E070E0F901E555FE4F9C
:101560008081882339F0CB01022E02C0880F991F99
:101570000A94E2F7482B2F5F3F4F2530310569F77A
:1015800020E030E060E270E0F901EF54FE4F80812E
:10159000882339F0CB01022E02C0880F991F0A94CC
:1015A000E2F7482B2F5F3F4F2330310569F748871B
:1015B000498520E030E061E070E0F901EC54FE4F35
:1015C0008081882339F0CB01022E02C0880F991F39
:1015D0000A94E2F7482B2F5F3F4F2430310569F71B
:1015E000498781E080934E01AFE4B1E0FE0132967D
:1015F00086E001900D928150E1F780914C0190912D
:101600004D01892B29F08FE780935301809354017A
:1016100088858093550189858093560180E001C0BB
:1016200081E029960FB6F894DEBF0FBECDBFCF91F3
:10163000DF911F910F9108950E94DA0990E08823AD
:1016400009F491E0892F08950E94DA09882399F41A
:101650008091B101882359F08091B201882339F03B
:1016600081E090E090934D0180934C010895109299
:101670004D0110924C0108958CEF90E0909306017B
:10168000809305010E94090DE5E0F1E092938293B9
:10169000CF01089520912F01253079F0222369F0A0
:1016A000892B31F0233049F082E080932F01089597
:1016B000213019F084E080932F010895CF92DF92BA
:1016C000EF92FF921F93DF93CF930F92CDB7DEB7C8
:1016D00085E080932F0110E08CE2C82E81E0D82EA7
:1016E0007E010894E11CF11C0E9420038CE291E031
:1016F000F6013197F1F70197D9F71982C70161E037
:1017000070E00E94CE08489711F481E004C01F5F8A
:101710001F3051F780E00F90CF91DF911F91FF9024
:10172000EF90DF90CF900895009741F0DC01E0E664
:10173000F1E089E001900D928150E1F7A9E6B1E076
:10174000E0E6F1E089E001900D928150E1F789E057
:1017500090E0089580E691E069E671E049E050E0AC
:101760000E940C0D08951F93DF93CF93CDB7DEB782
:10177000A6970FB6F894DEBF0FBECDBF1982CE017B
:10178000019661E070E00E94CE08883119F0109255
:101790002F016DC08091BF01882331F080912F010E
:1017A000853011F410922F018091BF01882319F424
:1017B00085E080932F0180912F018230E9F0843001
:1017C000A1F1882309F049C083E0898380E88A83F6
:1017D00081E08B83CE01049660E870E042E250E045
:1017E0000E94190DCE01019663E270E00E94CE08BE
:1017F000882399F184E02FC013E0198380EC8A8359
:101800008BE18B83CE01049661E070E040E250E012
:101810000E94190DCE01019663E270E00E94CE088D
:101820008823D9F010932F0118C083E0898380ECBE
:101830008A838BE18B8380E2FE013496DF011D9267
:101840008A95E9F7CE01019663E270E00E94CE0826
:10185000882319F081E080932F0181E08983CE01F4
:10186000019661E070E00E94CE08803211F08FEFA7
:10187000B0C019821A821B821C8240E020E030E056
:1018800061E070E0F901E855FE4F8081882339F06E
:10189000CB01022E02C0880F991F0A94E2F7482B51
:1018A0002F5F3F4F2430310569F720E030E060E1E1
:1018B00070E0F901EC54FE4F8081882339F0CB01B0
:1018C000022E02C0880F991F0A94E2F7482B2F5F5F
:1018D0003F4F2430310569F74B838091B20120E0FE
:1018E000811121E09C81922B8091B301811182E0D2
:1018F000892B8C83498120E030E060E870E0F901B9
:10190000E854FE4F8081882339F0CB01022E02C0BB
:10191000959587950A94E2F7482B2F5F3F4F283023
:10192000310569F749834A8120E030E060E870E0E2
:10193000F901E054FE4F8081882339F0CB01022E5B
:1019400002C0959587950A94E2F7482B2F5F3F4F89
:101950002830310569F74A8381E0809360018981ED
:101960008158809361018FE7982F941B90936201B7
:101970008093630180936401809365018093660185
:101980008B81809367019C81909368018091AC0169
:10199000882319F09460909368018091AD018823A9
:1019A00029F0809168018860809368018091AE0180
:1019B000882329F08091680180618093680180917B
:1019C000AF01882331F080916801806280936801C3
:1019D00080E0A6960FB6F894DEBF0FBECDBFCF91C4
:1019E000DF911F910895389A40980E94B30B089593
:1019F0008CEF90E090931C0180931B010E94090DD5
:101A0000EBE1F1E092938293CF01089582E190E0BF
:101A100008958CEE94E00895FB01DC0104C08D91E3
:101A20000190801921F441505040C8F7881B990B50
:101A30000895DC0101C06D9341505040E0F70895D6
:041A4000F894FFCF48
:101A44005AFFFF00000000010000000000240BDA30
:101A540009D109BB09B6091C0B00000000010000F4
:101A6400000000F30CB30BAA0B940B4A0B5E0B059E
:00000001FF
